:020000040000FA
:04080000D8EF07F036
:1008100003B213EF05F0F2B431EF05F09EB039EFFB
:1008200005F09EB241EF05F0F2A81AEF04F0F2B223
:1008300025EF04F0F2A620EF04F0F2B022EF04F06E
:1008400087EF07F0F296F290FF00CD90F2929EA013
:100850002FEF04F00101533F2FEF04F0542BAEC1F2
:10086000B2F1AFC1B3F1B0C1B4F1B1C1B5F1AAC138
:10087000AEF1ABC1AFF1ACC1B0F1ADC1B1F1A6C148
:10088000AAF1A7C1ABF1A8C1ACF1A9C1ADF1A2C158
:10089000A6F1A3C1A7F1A4C1A8F1A5C1A9F19EC168
:1008A000A2F19FC1A3F1A0C1A4F1A1C1A5F19AC178
:1008B0009EF19BC19FF19CC1A0F19DC1A1F196C188
:1008C0009AF197C19BF198C19CF199C19DF1CECF4E
:1008D00096F1CFCF97F153C198F154C199F1CF6AF6
:1008E000CE6A0101536B546B9E90CD800FBC0F8E6E
:1008F0000FBA7EEF04F00F8A87EF07F00F8C0FBE60
:10090000BAEF04F096C19AF197C19BF198C19CF19E
:1009100099C19DF19AC19EF19BC19FF19CC1A0F12B
:100920009DC1A1F19EC1A2F19FC1A3F1A0C1A4F1FB
:10093000A1C1A5F1A2C1A6F1A3C1A7F1A4C1A8F1CB
:10094000A5C1A9F1A6C1AAF1A7C1ABF1A8C1ACF19B
:10095000A9C1ADF1AAC1AEF1ABC1AFF1ACC1B0F16B
:10096000ADC1B1F1AEC1B2F1AFC1B3F1B0C1B4F13B
:10097000B1C1B5F101015E6B5F6B606B616B96514C
:100980005E2797515F2398516023995161239A51B3
:100990005E279B515F239C5160239D5161239E5193
:1009A0005E279F515F23A0516023A1516123A25173
:1009B0005E27A3515F23A4516023A5516123A65153
:1009C0005E27A7515F23A8516023A9516123AA5133
:1009D0005E27AB515F23AC516023AD516123AE5113
:1009E0005E27AF515F23B0516023B1516123B251F3
:1009F0005E27B3515F23B4516023B5516123D89072
:100A00000101613360335F335E33D890010161339C
:100A100060335F335E33D8900101613360335F33FD
:100A20005E3387EF07F00392ABB2AB98AB8803015C
:100A300003EE00F080517F0BE92604C0EFFF802B0E
:100A40008151805D700BD8A48B8200008051815D44
:100A5000700BD8A48B9281518019D8B4079087EF7E
:100A600007F0F2940101453F87EF07F0462B87EF2F
:100A700007F09E900101533F87EF07F0542B87EF5B
:100A800007F09E92040062A146EF05F0077C07ACD8
:100A900061EF05F0C274C2B45BEF05F0C3CFB3F5EC
:100AA000C4CFB4F50501D890B433B333D890B43380
:100AB000B33362EF05F0C3CF55F1C4CF56F162EF07
:100AC00005F0C28207B4CFEF05F047C14BF148C132
:100AD0004CF149C14DF14AC14EF15EC162F15FC1B5
:100AE00063F160C164F161C165F196C1B6F197C16E
:100AF000B7F198C1B8F199C1B9F19AC1BAF19BC1E6
:100B0000BBF19CC1BCF19DC1BDF19EC1BEF19FC1B5
:100B1000BFF1A0C1C0F1A1C1C1F1A2C1C2F1A3C185
:100B2000C3F1A4C1C4F1A5C1C5F1A6C1C6F1A7C155
:100B3000C7F1A8C1C8F1A9C1C9F1AAC1CAF1ABC125
:100B4000CBF1ACC1CCF1ADC1CDF1AEC1CEF1AFC1F5
:100B5000CFF1B0C1D0F1B1C1D1F1B2C1D2F1B3C1C5
:100B6000D3F1B4C1D4F1B5C1D5F1B3C5B5F5B4C5B0
:100B7000B6F5B5C5B7F5B6C5B8F5010155515B2752
:100B800056515C23E86A5D230E2ECFEF05F05CC161
:100B900057F15DC158F15B6B5C6B5D6B078E0201B9
:100BA000002F87EF07F03C0E006F05012F51000A60
:100BB000D8B486EF06F005012F51010AD8B410EF22
:100BC00006F005012F51020AD8B451EF06F00501D5
:100BD0002F51030AD8B451EF06F005012F51040A32
:100BE000D8B451EF06F005012F51050AD8B451EFE2
:100BF00006F005012F51060AD8B451EF06F00501A1
:100C00002F51070AD8B451EF06F005012F51320ACF
:100C1000D8B40EEF06F02F6B86EF06F086EF06F0E5
:100C2000050153671BEF06F054671BEF06F055678D
:100C30001BEF06F056671FEF06F086EF06F057C56C
:100C400000F158C501F159C502F15AC503F101017E
:100C5000010E046F000E056F000E066F000E076F89
:100C600025EC1FF000C157F501C158F502C159F537
:100C700003C15AF5006744EF06F0016744EF06F040
:100C8000026744EF06F0036786EF06F053C557F599
:100C900054C558F555C559F556C55AF50F8886EF10
:100CA00006F00501306757EF06F086EF06F00FBE3D
:100CB0006CEF06F010A071EF06F00101476768EFD6
:100CC00006F0486768EF06F0496768EF06F04A6784
:100CD0006CEF06F071EF06F007AE71EF06F083EFF0
:100CE00006F00501312F86EF06F03C0E316F302FF4
:100CF00086EF06F00101000E626FE00E636FA50E35
:100D0000646F010E656F0501306B0F880501626B22
:100D100033B78CEF06F062810CC100F10DC101F117
:100D20000EC102F10FC103F110C104F111C105F1AF
:100D300012C106F113C107F114C108F115C109F17F
:100D400016C10AF117C10BF135C134F100C10CF124
:100D500001C10DF102C10EF103C10FF104C110F187
:100D600005C111F106C112F107C113F108C114F157
:100D700009C115F10AC116F10BC117F134C135F1E2
:100D800001018A67CBEF06F08B67CBEF06F08C672B
:100D9000CBEF06F08D67CFEF06F0FFEF06F08EC1C8
:100DA00000F18FC101F190C102F191C103F1010184
:100DB000010E046F000E056F000E066F000E076F28
:100DC00025EC1FF000C18EF101C18FF102C190F13D
:100DD00003C191F10067F4EF06F00167F4EF06F04C
:100DE0000267F4EF06F00367FFEF06F08AC18EF1A9
:100DF0008BC18FF18CC190F18DC191F10F80D57EA7
:100E0000D5BE69D0D6CF47F1D7CF48F145C149F11A
:100E1000E86AE8CF4AF1109047C100F148C101F1FA
:100E200049C102F14AC103F101010A0E046F000E2B
:100E3000056F000E066F000E076F25EC1FF003AF65
:100E40001080010154A731EF07F00F9A0F9C0F9EFD
:100E50000101000E5E6F600E5F6F3D0E606F080E49
:100E6000616F010147BF41EF07F0486741EF07F0AD
:100E7000496741EF07F04A6741EF07F0F28866EFF4
:100E800007F0F2985E6B5F6B606B616B966B976BB4
:100E9000986B996B9A6B9B6B9C6B9D6B9E6B9F6B1E
:100EA000A06BA16BA26BA36BA46BA56BA66BA76BCE
:100EB000A86BA96BAA6BAB6BAC6BAD6BAE6BAF6B7E
:100EC000B06BB16BB26BB36BB46BB56BD76AD66AF0
:100ED0000101456B466B0CC100F10DC101F10EC162
:100EE00002F10FC103F110C104F111C105F112C1EA
:100EF00006F113C107F114C108F115C109F116C1BA
:100F00000AF117C10BF135C134F187EF07F002C0C8
:100F1000E0FF005001C0D8FF1000A6B28DEF07F02F
:100F20000CC0A9FF0BC0A8FFA69EA69CA684F29E9B
:100F3000550EA76EAA0EA76EA682F28EA694A6B232
:100F40009FEF07F00C2A1200A96EA69EA69CA68011
:100F5000A8500C2A120004012C0E826F92EC0AF0A9
:100F600020EC20F00C50A4EC07F0E8CF00F10C507E
:100F7000A4EC07F0E8CF01F101AFC4EF07F00101E5
:100F8000FF0E026FFF0E036FC3EC1FF02967D0EF57
:100F900007F00401200E826F92EC0AF0D5EF07F003
:100FA00004012D0E826F92EC0AF0EDEC1DF01200A0
:100FB000076A0F6A106A0F010D0EC16E860EC06EB1
:100FC000030EC26E0F01680E896E130E926E080E2C
:100FD0008A6EF30E936E8B6A900E946EF18EF19E74
:100FE0000E6A01015B6B5C6B5D6B576B586BF29A21
:100FF0000101476B486B496B4A6B4B6B4C6B4D6BFC
:101000004E6B4F6B506B516B526B456B466BD76A97
:10101000D66A0F01280ED56EF28A9D90B00ECD6E65
:1010200001015E6B5F6B606B616B626B636B646B2A
:10103000656B666B676B686B696B536B546BCF6AE0
:10104000CE6A0F9A0F9C0F9E9D80760ECA6E9D826F
:1010500002013C0E006FCC6A160EA4EC07F0E8CF3C
:1010600000F1170EA4EC07F0E8CF01F1180EA4EC84
:1010700007F0E8CF02F1190EA4EC07F0E8CF03F176
:10108000010103AF5EEF08F020EC20F0160E0C6EAD
:1010900000C10BF08DEC07F0170E0C6E01C10BF0C8
:1010A0008DEC07F0180E0C6E02C10BF08DEC07F002
:1010B000190E0C6E03C10BF08DEC07F000C18AF124
:1010C00001C18BF102C18CF103C18DF100C18EF120
:1010D00001C18FF102C190F103C191F11A0EA4EC8C
:1010E00007F0E8CF00F11B0EA4EC07F0E8CF01F108
:1010F0001C0EA4EC07F0E8CF02F11D0EA4EC07F0E3
:10110000E8CF03F1010103AFB4EF08F020EC20F0C9
:101110001A0E0C6E00C10BF08DEC07F01B0E0C6E5E
:1011200001C10BF08DEC07F01C0E0C6E02C10BF030
:101130008DEC07F01D0E0C6E03C10BF08DEC07F06B
:101140001A0EA4EC07F0E8CF00F11B0EA4EC07F098
:10115000E8CF01F11C0EA4EC07F0E8CF02F11D0E60
:10116000A4EC07F0E8CF03F100C192F101C193F1C3
:1011700002C194F103C195F1240EAC6E900EAB6EDA
:10118000240EAC6E080EB86E000EB06E1F0EAF6E61
:101190000401806B816B0F01900EAB6E0F019D8A75
:1011A0000301806B816BC26B8B9264EC25F064EC65
:1011B00025F0C0EC26F045EC23F0200EA4EC07F05F
:1011C000E8CF2FF505012F51FF0AD8A4EFEF08F063
:1011D0002F6B200E0C6E2FC50BF08DEC07F0050168
:1011E000010E306F3C0E316F250EA4EC07F0E8CFF6
:1011F00000F1260EA4EC07F0E8CF01F1270EA4ECD5
:1012000007F0E8CF02F1280EA4EC07F0E8CF03F1D5
:10121000010103AF26EF09F020EC20F0250E0C6E43
:1012200000C10BF08DEC07F0260E0C6E01C10BF027
:101230008DEC07F0270E0C6E02C10BF08DEC07F061
:10124000280E0C6E03C10BF08DEC07F000C153F5B6
:1012500001C154F502C155F503C156F500C157F55A
:1012600001C158F502C159F503C15AF5290EA4EC84
:1012700007F0E8CF5BF505015C515B5DD8A05BC56D
:101280005CF505012F51020A0EE181B853EF09F018
:1012900005015C2F50EF09F05BC55CF553EF09F0D9
:1012A00081BAFFEF26F0210EA4EC07F0E8CF00F1A1
:1012B000220EA4EC07F0E8CF01F1230EA4EC07F016
:1012C000E8CF02F1240EA4EC07F0E8CF03F101010E
:1012D00003AF99EF09F020EC20F0210E0C6E00C155
:1012E0000BF08DEC07F0220E0C6E01C10BF08DECB3
:1012F00007F0230E0C6E02C10BF08DEC07F0240EEC
:101300000C6E03C10BF08DEC07F0210EA4EC07F07E
:10131000E8CF00F1220EA4EC07F0E8CF01F1230E94
:10132000A4EC07F0E8CF02F1240EA4EC07F0E8CF1C
:1013300003F100C15DF501C15EF502C15FF503C1B6
:1013400060F57CEC22F03EEC21F08EEC20F0050103
:101350002F51030A12E005012F51040A1DE0050177
:101360002F51050A24E005012F51060A32E005013C
:101370002F51070A38E0FCEF09F0ACC500F101017C
:101380000F0E001701010051000A36E00101005163
:10139000050A32E0F9EF09F0ACC500F101010F0ECA
:1013A000001701010051000A27E0F9EF09F00501DB
:1013B000AC51000A21E00501AC51150A1DE0050100
:1013C000AC51300A19E00501AC51450A15E0F9EFBE
:1013D00009F00501AC51000A0FE00501AC51300ADB
:1013E0000BE0F9EF09F00501AC51000A05E0F9EF57
:1013F00009F081BAFFEF26F007900001F28EF28C1F
:1014000007B06EEF1CF00FB04FEF17F00FB813EFEF
:1014100011F00301805181197F0BD8B46EEF1CF0DD
:1014200013EE00F081517F0BE126812BE7CFE8FF1F
:10143000E00BD8B46EEF1CF023EE82F0C2513F0BEC
:10144000D926E7CFDFFFC22BDF50780AD8A46EEF92
:101450001CF007808EC100F18FC101F190C102F133
:1014600091C103F10101040E046F000E056F000E1F
:10147000066F000E076F25EC1FF000AF49EF0AF072
:101480000101030E8E6F000E8F6F000E906F000E25
:10149000916F03018251720AD8B44FEF17F0825155
:1014A000520AD8B44FEF17F08251750AD8B44FEFF3
:1014B00017F08251630AD8B42AEF19F08251690AF1
:1014C000D8B40AEF14F082517A0AD8B41DEF15F09F
:1014D0008251490AD8B4A9EF13F08251500AD8B406
:1014E000C7EF12F08251700AD8B40AEF13F082519C
:1014F000540AD8B435EF13F08251740AD8B47BEF94
:1015000013F08251730AD8B47FEF16F08251530A58
:10151000D8B4E4EF16F082514C0AD8B4A6EF0AF022
:101520005FEF19F0040114EE00F080517F0BE1260B
:1015300082C4E7FF802B120004010D0E826F92EC33
:101540000AF00A0E826F92EC0AF012000301835136
:10155000300AD8B40BEF0EF003018351310AD8B42E
:1015600019EF0FF003018351320AD8B487EF0FF05F
:1015700003018351330AD8B497EF0FF0030183516D
:10158000340AD8B4A7EF0FF003018351350AD8B459
:1015900018EF11F003018351360AD8B446EF11F069
:1015A00003018351370AD8B46DEF0DF00301835165
:1015B000460AD8B46CEF10F0030183514D0AD8B439
:1015C000E6EF0BF0030183516D0AD8B400EF0CF085
:1015D000030183515A0AD8B493EF0EF003018351EB
:1015E000490AD8B446EF12F003018351500AD8B427
:1015F00078EF11F003018351540AD8B4F1EF11F0E0
:1016000003018351630AD8B420EF0CF00301835126
:10161000430AD8B418EF0DF003018351730AD8B40C
:101620001EEF0CF003018351610AD8B433EF0BF0C5
:1016300003018351650AD8B45BEF0EF003018351B7
:10164000450AD8B469EF0EF003018351620AD8B499
:1016500077EF0EF003018351420AD8B485EF0EF004
:10166000D8A45FEF19F004014C0E826F92EC0AF0DF
:101670000401610E826F92EC0AF03EEC21F004014D
:101680002C0E826F92EC0AF020EC20F0ABC500F13A
:101690000101C3EC1FF031C182F40401300E822736
:1016A00092EC0AF032C182F40401300E822792ECEF
:1016B0000AF033C182F40401300E822792EC0AF062
:1016C00004012C0E826F92EC0AF020EC20F0ACC5E5
:1016D00000F10101C3EC1FF031C182F40401300EAE
:1016E000822792EC0AF032C182F40401300E822784
:1016F00092EC0AF033C182F40401300E822792EC9E
:101700000AF004012C0E826F92EC0AF020EC20F01B
:10171000ADC500F10101C3EC1FF031C182F4040139
:10172000300E822792EC0AF032C182F40401300EAE
:10173000822792EC0AF033C182F40401300E822732
:1017400092EC0AF004012C0E826F92EC0AF020EC6D
:1017500020F0AEC500F10101C3EC1FF031C182F4ED
:101760000401300E822792EC0AF032C182F40401A7
:10177000300E822792EC0AF033C182F40401300E5D
:10178000822792EC0AF004012C0E826F92EC0AF090
:1017900020EC20F0B3C500F10101C3EC1FF031C112
:1017A00082F40401300E822792EC0AF032C182F4F6
:1017B0000401300E822792EC0AF033C182F4040156
:1017C000300E822792EC0AF074EF11F061EC20F0F9
:1017D00084C333F16EEC20F0E5EC1FF0200E0C6EAC
:1017E00000C10BF08DEC07F000C12FF505012F5162
:1017F000000A06E005012F51010A02E0E4EC21F0A5
:1018000004014C0E826F92EC0AF004014D0E826FBF
:1018100092EC0AF004012C0E826F92EC0AF020EC9C
:1018200020F02FC500F1C3EC1FF033C182F4040196
:10183000300E822792EC0AF074EF11F0FFEF26F0E1
:1018400004014C0E826F92EC0AF00401630E826F69
:1018500092EC0AF08EEC20F004012C0E826F92ECD8
:101860000AF035EC0CF074EF11F020EC20F0B1C56B
:1018700000F10101003B0F0E0017C3EC1FF033C154
:1018800082F40401300E822792EC0AF0B1C500F117
:1018900001010F0E01010017C3EC1FF033C182F4E8
:1018A0000401300E822792EC0AF004012D0E826FA3
:1018B00092EC0AF0B0C500F10101003B0F0E0017D9
:1018C000C3EC1FF033C182F40401300E822792EC86
:1018D0000AF0B0C500F101010F0E01010017C3ECC1
:1018E0001FF033C182F40401300E822792EC0AF01B
:1018F00004012D0E826F92EC0AF0AFC500F10101D8
:10190000003B0F0E0017C3EC1FF033C182F404013B
:10191000300E822792EC0AF0AFC500F101010F0EE4
:1019200001010017C3EC1FF033C182F40401300E33
:10193000822792EC0AF00401200E826F92EC0AF0EA
:10194000AEC500F10F0E01010017C3EC1FF033C14B
:1019500082F40401300E822792EC0AF00401200E7A
:10196000826F92EC0AF0ADC500F101010101003B6C
:101970000F0E0017C3EC1FF033C182F40401300EC8
:10198000822792EC0AF0ADC500F101010F0E0101B2
:101990000017C3EC1FF033C182F40401300E82271C
:1019A00092EC0AF004013A0E826F92EC0AF0ACC598
:1019B00000F10101003B0F0E0017C3EC1FF033C113
:1019C00082F40401300E822792EC0AF0ACC500F1DB
:1019D00001010F0E01010017C3EC1FF033C182F4A7
:1019E0000401300E822792EC0AF004013A0E826F55
:1019F00092EC0AF0ABC500F10101003B0F0E00179D
:101A0000C3EC1FF033C182F40401300E822792EC44
:101A10000AF0ABC500F101010F0E0017C3EC1FF077
:101A200033C182F40401300E822792EC0AF01200D6
:101A300084C3E8FF0F0BE83AE8CFB1F585C3E8FFB0
:101A40000F0B0501B11387C3E8FF0F0BE83AE8CF8E
:101A5000B0F588C3E8FF0F0B0501B0138AC3E8FF98
:101A60000F0BE83AE8CFAFF58BC3E8FF0F0B05018A
:101A7000AF138DC3E8FF0F0BE8CFAEF58FC3E8FFC0
:101A80000F0BE83AE8CFADF590C3E8FF0F0B050167
:101A9000AD1392C3E8FF0F0BE83AE8CFACF593C360
:101AA000E8FF0F0B0501AC1395C3E8FF0F0BE83AF5
:101AB000E8CFABF596C3E8FF0F0B0501AB13EDECD8
:101AC00020F004014C0E826F92EC0AF00401430EE8
:101AD000826F92EC0AF02AEF0CF0078404014C0E9E
:101AE000826F92EC0AF00401370E826F92EC0AF0DA
:101AF00004012C0E826F92EC0AF005012E51130A9C
:101B000006E005012E51170A0DE008EF0EF0010165
:101B1000000E006F000E016F100E026F000E036FBB
:101B20009BEF0DF00101000E006F000E016F000E23
:101B3000026F010E036FC3EC1FF02AC182F404018F
:101B4000300E822792EC0AF02BC182F40401300E91
:101B5000822792EC0AF02CC182F40401300E822715
:101B600092EC0AF02DC182F40401300E822792EC2F
:101B70000AF02EC182F40401300E822792EC0AF0A2
:101B80002FC182F40401300E822792EC0AF030C19A
:101B900082F40401300E822792EC0AF031C182F403
:101BA0000401300E822792EC0AF032C182F4040163
:101BB000300E822792EC0AF033C182F40401300E19
:101BC000822792EC0AF004012C0E826F92EC0AF04C
:101BD0000101100E006F000E016F000E026F000E6B
:101BE000036FC3EC1FF031C182F40401300E822771
:101BF00092EC0AF032C182F40401300E822792EC9A
:101C00000AF033C182F40401300E822792EC0AF00C
:101C1000079474EF11F00784C0EC26F020EC20F05C
:101C20002DC500F1C3EC1FF004014C0E826F92EC45
:101C30000AF00401300E826F92EC0AF004012C0EBF
:101C4000826F92EC0AF031C182F40401300E8227D7
:101C500092EC0AF032C182F40401300E822792EC39
:101C60000AF033C182F40401300E822792EC0AF0AC
:101C700004012C0E826F92EC0AF020EC20F02EC5AD
:101C800000F1C3EC1FF031C182F40401300E822751
:101C900092EC0AF032C182F40401300E822792ECF9
:101CA0000AF033C182F40401300E822792EC0AF06C
:101CB000079474EF11F004014C0E826F92EC0AF05D
:101CC0000401650E826F92EC0AF0CDEC22F074EF05
:101CD00011F004014C0E826F92EC0AF00401450EE3
:101CE000826F92EC0AF0EAEC22F074EF11F004013A
:101CF0004C0E826F92EC0AF00401620E826F92EC3D
:101D00000AF024EC23F074EF11F004014C0E826F02
:101D100092EC0AF00401420E826F92EC0AF007EC9A
:101D200023F074EF11F004014C0E826F92EC0AF074
:101D300004015A0E826F92EC0AF004012C0E826F9D
:101D400092EC0AF0C0EC26F020EC20F005012E51B8
:101D5000130A06E005012E51170A0DE0C4EF0EF03C
:101D60000101000E006F000E016F100E026F000ED9
:101D7000036FC4EF0EF00101000E006F000E016F43
:101D8000000E026F010E036F0101100E046F000EB2
:101D9000056F000E066F000E076F56EC1FF0C3ECC8
:101DA0001FF02AC182F40401300E822792EC0AF05F
:101DB0002BC182F40401300E822792EC0AF02CC170
:101DC00082F40401300E822792EC0AF02DC182F4D5
:101DD0000401300E822792EC0AF02EC182F4040135
:101DE000300E822792EC0AF02FC182F40401300EEB
:101DF000822792EC0AF030C182F40401300E82276F
:101E000092EC0AF031C182F40401300E822792EC88
:101E10000AF032C182F40401300E822792EC0AF0FB
:101E200033C182F40401300E822792EC0AF074EF81
:101E300011F0078404014C0E826F92EC0AF0040149
:101E4000310E826F92EC0AF004012C0E826F92EC3C
:101E50000AF025C500F126C501F127C502F128C504
:101E600003F10101100E046F000E056F000E066FE6
:101E7000000E076F56EC1FF0C3EC1FF02AC182F46E
:101E80000401300E822792EC0AF02BC182F4040187
:101E9000300E822792EC0AF02CC182F40401300E3D
:101EA000822792EC0AF02DC182F40401300E8227C1
:101EB00092EC0AF02EC182F40401300E822792ECDB
:101EC0000AF02FC182F40401300E822792EC0AF04E
:101ED00030C182F40401300E822792EC0AF031C145
:101EE00082F40401300E822792EC0AF032C182F4AF
:101EF0000401300E822792EC0AF033C182F404010F
:101F0000300E822792EC0AF0079474EF11F00784E8
:101F100004014C0E826F92EC0AF00401320E826FC3
:101F200092EC0AF01AEC25F0079474EF11F0078494
:101F300004014C0E826F92EC0AF00401330E826FA2
:101F400092EC0AF077EC25F0079424EF0FF0078469
:101F500004014C0E826F92EC0AF00401340E826F81
:101F600092EC0AF004012C0E826F92EC0AF061EC04
:101F700020F084C32AF185C32BF186C32CF187C3DB
:101F80002DF188C32EF189C32FF18AC330F18BC3A1
:101F900031F18CC332F18DC333F10101296B6EEC49
:101FA00020F0E5EC1FF0100E046F000E056F000E20
:101FB000066F000E076F36EC1FF000C121F501C15E
:101FC00022F502C123F503C124F573EC26F034C5D4
:101FD000ABF535C5ACF536C5ADF537C5AEF538C58D
:101FE000AFF539C5B0F53AC5B1F535EC0CF00401E3
:101FF0002C0E826F92EC0AF03BC500F13CC501F15A
:102000003DC502F13EC503F10101000E046F000E53
:10201000056F010E066F000E076F56EC1FF0C3EC44
:102020001FF0296716EF10F01BEF10F004012D0EC2
:10203000826F92EC0AF030C182F40401300E8227E4
:1020400092EC0AF031C182F40401300E822792EC46
:102050000AF004012E0E826F92EC0AF032C182F473
:102060000401300E822792EC0AF033C182F404019D
:10207000300E822792EC0AF004012C0E826F92EC53
:102080000AF020EC20F03FC500F140C501F189ECD9
:102090001AF004012C0E826F92EC0AF020EC20F072
:1020A00041C500F1C3EC1FF031C182F40401300ED0
:1020B000822792EC0AF032C182F40401300E8227AA
:1020C00092EC0AF033C182F40401300E822792ECC4
:1020D0000AF0079474EF11F061EC20F085C32AF147
:1020E00086C32BF187C32CF188C32DF189C32EF150
:1020F0008AC32FF18BC330F18CC331F18DC332F120
:102100008EC333F10101296B6EEC20F0E5EC1FF07A
:102110000101010E046F000E056F000E066F000E28
:10212000076F25EC1FF0100E046F000E056F000EF8
:10213000066F000E076F36EC1FF000C129F501C1D4
:102140002AF502C12BF503C12CF5A3EC24F0040100
:102150004C0E826F92EC0AF00401460E826F92ECF4
:102160000AF004012C0E826F92EC0AF025C500F1F2
:1021700026C501F127C502F128C503F10101100EA2
:10218000046F000E056F000E066F000E076F56EC11
:102190001FF0C3EC1FF02AC182F40401300E822725
:1021A00092EC0AF02BC182F40401300E822792ECEB
:1021B0000AF02CC182F40401300E822792EC0AF05E
:1021C0002DC182F40401300E822792EC0AF02EC158
:1021D00082F40401300E822792EC0AF02FC182F4BF
:1021E0000401300E822792EC0AF030C182F404011F
:1021F000300E822792EC0AF031C182F40401300ED5
:10220000822792EC0AF032C182F40401300E822758
:1022100092EC0AF033C182F40401300E822792EC72
:102220000AF074EF11F00F9877EC25F05FEF19F0DA
:1022300004014C0E826F92EC0AF00401350E826F9D
:1022400092EC0AF004012C0E826F92EC0AF020EC62
:1022500020F00784B5C500F10794C3EC1FF031C12D
:1022600082F40401300E822792EC0AF032C182F42B
:102270000401300E822792EC0AF033C182F404018B
:10228000300E822792EC0AF074EF11F03AEC25F050
:1022900020EC20F033C500F1C3EC1FF004014C0E1C
:1022A000826F92EC0AF00401360E826F92EC0AF013
:1022B00004012C0E826F92EC0AF031C182F4040109
:1022C000300E822792EC0AF032C182F40401300E03
:1022D000822792EC0AF033C182F40401300E822787
:1022E00092EC0AF074EF11F09CEC0AF05FEF19F039
:1022F00004014C0E826F92EC0AF00401500E826FC2
:1023000092EC0AF004012C0E826F92EC0AF085C365
:102310002AF186C32BF187C32CF188C32DF189C321
:102320002EF18AC32FF18BC330F18CC331F18DC3F1
:1023300032F18EC333F101016EEC20F0E5EC1FF0B9
:1023400003018451530A0DE0030184514D0A38E022
:102350000401780E826F92EC0AF09CEC0AF05FEFB9
:1023600019F00401530E826F92EC0AF0250E0C6EE8
:1023700000C10BF08DEC07F0260E0C6E01C10BF0C6
:102380008DEC07F0270E0C6E02C10BF08DEC07F000
:10239000280E0C6E03C10BF08DEC07F000C153F555
:1023A00001C154F502C155F503C156F500C157F5F9
:1023B00001C158F502C159F503C15AF555EF12F0A4
:1023C00004014D0E826F92EC0AF0290E0C6E00C1D2
:1023D0000BF08DEC07F000C15BF500C15CF555EF2B
:1023E00012F004014C0E826F92EC0AF00401540EBC
:1023F000826F92EC0AF004012C0E826F92EC0AF0CC
:1024000084C32AF185C32BF186C32CF187C32DF138
:1024100088C32EF189C32FF18AC330F18BC331F108
:102420008DC332F18EC333F101016EEC20F0E5EC87
:102430001FF00101000E046F000E056F010E066F04
:10244000000E076F36EC1FF0210E0C6E00C10BF072
:102450008DEC07F0220E0C6E01C10BF08DEC07F035
:10246000230E0C6E02C10BF08DEC07F0240E0C6EE7
:1024700003C10BF08DEC07F000C15DF501C15EF505
:1024800002C15FF503C160F555EF12F004014C0E77
:10249000826F92EC0AF00401490E826F92EC0AF00E
:1024A00004012C0E826F92EC0AF0250EA4EC07F0CA
:1024B000E8CF00F1260EA4EC07F0E8CF01F1270EDB
:1024C000A4EC07F0E8CF02F1280EA4EC07F0E8CF67
:1024D00003F1C3EC1FF0A6EC1DF00401730E826F34
:1024E00092EC0AF004012C0E826F92EC0AF020ECC0
:1024F00020F0290EA4EC07F0E8CF00F1C3EC1FF0A8
:10250000A6EC1DF00401730E826F92EC0AF0040138
:102510002C0E826F92EC0AF057C500F158C501F1FC
:1025200059C502F15AC503F1C3EC1FF0A6EC1DF02A
:102530000401730E826F92EC0AF004012C0E826F7C
:1025400092EC0AF020EC20F05CC500F1C3EC1FF027
:10255000A6EC1DF004016D0E826F92EC0AF00401EE
:102560002C0E826F92EC0AF05DC500F15EC501F1A0
:102570005FC502F160C503F17AEC19F004012C0E7D
:10258000826F92EC0AF09CEC0AF05FEF19F083C3C3
:102590002AF184C32BF185C32CF186C32DF187C3A7
:1025A0002EF188C32FF189C330F18AC331F18BC377
:1025B00032F18CC333F101016EEC20F0E5EC1FF039
:1025C000160E0C6E00C10BF08DEC07F0170E0C6EA2
:1025D00001C10BF08DEC07F0180E0C6E02C10BF070
:1025E0008DEC07F0190E0C6E03C10BF08DEC07F0AB
:1025F00000C18AF101C18BF102C18CF103C18DF1DF
:1026000000C18EF101C18FF102C190F103C191F1BE
:10261000A9EF13F083C32AF184C32BF185C32CF1F6
:1026200086C32DF187C32EF188C32FF189C330F102
:102630008AC331F18BC332F18CC333F101016EECEB
:1026400020F0E5EC1FF000C18AF101C18BF102C15D
:102650008CF103C18DF100C18EF101C18FF102C176
:1026600090F103C191F1A9EF13F083C32AF184C360
:102670002BF185C32CF186C32DF187C32EF188C3BE
:102680002FF189C330F18AC331F18CC332F18DC38C
:1026900033F101016EEC20F0E5EC1FF00101000EBA
:1026A000046F000E056F010E066F000E076F36EC0B
:1026B0001FF01A0E0C6E00C10BF08DEC07F01B0E14
:1026C0000C6E01C10BF08DEC07F01C0E0C6E02C1FC
:1026D0000BF08DEC07F01D0E0C6E03C10BF08DECB2
:1026E00007F000C192F101C193F102C194F103C15D
:1026F00095F1A9EF13F083C32AF184C32BF185C3AD
:102700002CF186C32DF187C32EF188C32FF189C325
:1027100030F18AC331F18CC332F18DC333F1010141
:102720006EEC20F0E5EC1FF00101000E046F000ECE
:10273000056F010E066F000E076F36EC1FF000C12B
:1027400092F101C193F102C194F103C195F1A9EF96
:1027500013F0160EA4EC07F0E8CF00F1170EA4EC6E
:1027600007F0E8CF01F1180EA4EC07F0E8CF02F172
:10277000190EA4EC07F0E8CF03F1C3EC1FF0A6ECB0
:102780001DF00401730E826F92EC0AF004012C0E0E
:10279000826F92EC0AF08AC100F18BC101F18CC109
:1027A00002F18DC103F1C3EC1FF0A6EC1DF0040192
:1027B000730E826F92EC0AF004012C0E826F92EC81
:1027C0000AF01A0EA4EC07F0E8CF00F11B0EA4ECFF
:1027D00007F0E8CF01F11C0EA4EC07F0E8CF02F1FE
:1027E0001D0EA4EC07F0E8CF03F17AEC19F0040118
:1027F0002C0E826F92EC0AF092C100F193C101F1AC
:1028000094C102F195C103F17AEC19F09CEC0AF045
:102810005FEF19F00401690E826F92EC0AF0040177
:102820002C0E826F92EC0AF00101040E006F000E74
:10283000016F000E026F000E036FC3EC1FF02CC17E
:1028400082F40401300E822792EC0AF02DC182F44A
:102850000401300E822792EC0AF02EC182F40401AA
:10286000300E822792EC0AF02FC182F40401300E60
:10287000822792EC0AF030C182F40401300E8227E4
:1028800092EC0AF031C182F40401300E822792ECFE
:102890000AF032C182F40401300E822792EC0AF071
:1028A00033C182F40401300E822792EC0AF0040155
:1028B0002C0E826F92EC0AF00101060E006F000EE2
:1028C000016F000E026F000E036FC3EC1FF02CC1EE
:1028D00082F40401300E822792EC0AF02DC182F4BA
:1028E0000401300E822792EC0AF02EC182F404011A
:1028F000300E822792EC0AF02FC182F40401300ED0
:10290000822792EC0AF030C182F40401300E822753
:1029100092EC0AF031C182F40401300E822792EC6D
:102920000AF032C182F40401300E822792EC0AF0E0
:1029300033C182F40401300E822792EC0AF00401C4
:102940002C0E826F92EC0AF00101220E006F000E35
:10295000016F000E026F000E036FC3EC1FF02CC15D
:1029600082F40401300E822792EC0AF02DC182F429
:102970000401300E822792EC0AF02EC182F4040189
:10298000300E822792EC0AF02FC182F40401300E3F
:10299000822792EC0AF030C182F40401300E8227C3
:1029A00092EC0AF031C182F40401300E822792ECDD
:1029B0000AF032C182F40401300E822792EC0AF050
:1029C00033C182F40401300E822792EC0AF0040134
:1029D0002C0E826F92EC0AF0200EF86EF76AF66AFF
:1029E00004010900F5CF82F492EC0AF00900F5CF5A
:1029F00082F492EC0AF00900F5CF82F492EC0AF02E
:102A00000900F5CF82F492EC0AF00900F5CF82F4C8
:102A100092EC0AF00900F5CF82F492EC0AF009007A
:102A2000F5CF82F492EC0AF00900F5CF82F492EC33
:102A30000AF09CEC0AF05FEF19F08351630AD8A406
:102A40005FEF19F08451610AD8A45FEF19F0855146
:102A50006C0AD8A45FEF19F08651410A42E0865112
:102A6000440A1BE08651420AD8B484EF15F086511F
:102A7000350AD8B4E9EF1AF08651360AD8B43EEFD9
:102A80001BF08651370AD8B4A7EF1BF08651380ADD
:102A9000D8B405EF1CF05FEF19F00798079A04010E
:102AA0007A0E826F92EC0AF00401780E826F92EC3B
:102AB0000AF00401640E826F92EC0AF081A868EFBC
:102AC00015F00401550E826F92EC0AF06DEF15F0CF
:102AD00004014C0E826F92EC0AF09CEC0AF05FEF5E
:102AE00019F00788079A04017A0E826F92EC0AF0B7
:102AF0000401410E826F92EC0AF00401610E826FB4
:102B000092EC0AF05EEF15F00798078A04017A0E3E
:102B1000826F92EC0AF00401420E826F92EC0AF08E
:102B20000401610E826F92EC0AF05EEF15F0010174
:102B30006667A2EF15F06767A2EF15F06867A2EF6E
:102B400015F06967BAEF15F04F67AEEF15F05067F3
:102B5000AEEF15F05167AEEF15F05267BAEF15F012
:102B60000101000E006F000E016F000E026F000EDB
:102B7000036F12000101620E046F010E056F000E5B
:102B8000066F000E076F66C100F167C101F168C1F1
:102B900002F169C103F125EC1FF003BF3EEF16F00F
:102BA0000101000E046FA80E056F550E066F020E90
:102BB000076F66C100F167C101F168C102F169C127
:102BC00003F166C186F167C187F168C188F169C107
:102BD00089F125EC1FF003BFF7EF15F00101000E9E
:102BE000866FA80E876F550E886F020E896F0E0EC6
:102BF000A4EC07F0E8CF18F10F0EA4EC07F0E8CF33
:102C000019F1100EA4EC07F0E8CF1AF1110EA4ECA4
:102C100007F0E8CF1BF16EEC1EF086C104F187C10E
:102C200005F188C106F189C107F125EC1FF0078283
:102C300032EC1EF06EEC1EF0079232EC1EF086C1F4
:102C400000F187C101F188C102F189C103F1079246
:102C500032EC1EF0CC0E046FE00E056F870E066F8F
:102C6000050E076F25EC1FF000C118F101C119F125
:102C700002C11AF103C11BF176EF16F00101800EBB
:102C8000006F1A0E016F060E026F000E036F4FC128
:102C900004F150C105F151C106F152C107F125EC13
:102CA0001FF003AF57EF16F020EC20F012000E0ECD
:102CB000A4EC07F0E8CF18F10F0EA4EC07F0E8CF72
:102CC00019F1100EA4EC07F0E8CF1AF1110EA4ECE4
:102CD00007F0E8CF1BF14FC100F150C101F151C124
:102CE00002F152C103F1078232EC1EF018C100F16B
:102CF00019C101F11AC102F11BC103F11200040153
:102D0000730E826F92EC0AF004012C0E826F92EC2B
:102D10000AF0078462C166F163C167F164C168F1BA
:102D200065C169F14BC14FF14CC150F14DC151F139
:102D30004EC152F157C159F158C15AF10794A5EC4F
:102D400016F09CEC0AF05FEF19F066C100F167C164
:102D500001F168C102F169C103F10101C3EC1FF087
:102D6000A6EC1DF00401630E826F92EC0AF00401E0
:102D70002C0E826F92EC0AF04FC100F150C101F1AC
:102D800051C102F152C103F10101C3EC1FF0A6ECE5
:102D90001DF00401660E826F92EC0AF004012C0E05
:102DA000826F92EC0AF020EC20F059C100F15AC178
:102DB00001F10101C3EC1FF0A6EC1DF00401740E3B
:102DC000826F92EC0AF0120010820401530E826F9F
:102DD00092EC0AF004012C0E826F92EC0AF083C38D
:102DE0002AF184C32BF185C32CF186C32DF187C34F
:102DF0002EF188C32FF189C330F18AC331F18BC31F
:102E000032F18CC333F101016EEC20F0E5EC1FF0E0
:102E100000C166F101C167F102C168F103C169F146
:102E20008EC32AF18FC32BF190C32CF191C32DF1E6
:102E300092C32EF193C32FF194C330F195C331F1B6
:102E400096C332F197C333F101016EEC20F0E5EC4B
:102E50001FF000C14FF101C150F102C151F103C196
:102E600052F161EC20F099C32FF19AC330F19BC36A
:102E700031F19CC332F19DC333F101016EEC20F0BE
:102E8000E5EC1FF000C159F101C15AF1A5EC16F0B3
:102E900004012C0E826F92EC0AF056EF17F082516B
:102EA000520A03E10F8256EF17F00F928251750A12
:102EB00003E110845DEF17F010948251550A03E18D
:102EC000108664EF17F01096078410B2C1EF17F068
:102ED00010A4ADEF17F0B6C166F1B7C167F1B8C184
:102EE00068F1B9C169F1BAC16AF1BBC16BF1BCC18A
:102EF0006CF1BDC16DF1BEC16EF1BFC16FF1C0C15A
:102F000070F1C1C171F1C2C172F1C3C173F1C4C129
:102F100074F1C5C175F1C6C176F1C7C177F1C8C1F9
:102F200078F1C9C179F1CAC17AF1CBC17BF1CCC1C9
:102F30007CF1CDC17DF1CEC17EF1CFC17FF1D0C199
:102F400080F1D1C181F1D2C182F1D3C183F1D4C169
:102F500084F1D5C185F1B5EF17F062C166F163C1A7
:102F600067F164C168F165C169F14BC14FF14CC1B2
:102F700050F14DC151F14EC152F157C159F158C1F3
:102F80005AF107940FA0E3EF17F001019267D0EF19
:102F900017F09367D0EF17F09467D0EF17F09567AD
:102FA000D4EF17F0E3EF17F097EC15F092C104F1AE
:102FB00093C105F194C106F195C107F125EC1FF00D
:102FC00003BF27EF19F097EC15F00101000E046F15
:102FD000000E056F010E066F000E076F56EC1FF016
:102FE00010A4FAEF17F00401750E826F92EC0AF04C
:102FF000FFEF17F00401720E826F92EC0AF00401E9
:103000002C0E826F92EC0AF0C3EC1FF029670EEFD2
:1030100018F00401200E826F11EF18F004012D0E3C
:10302000826F92EC0AF030C182F40401300E8227E4
:1030300092EC0AF031C182F40401300E822792EC46
:103040000AF004012E0E826F92EC0AF032C182F473
:103050000401300E822792EC0AF033C182F404019D
:10306000300E822792EC0AF004016D0E826F92EC12
:103070000AF004012C0E826F92EC0AF04FC100F1AD
:1030800050C101F151C102F152C103F10101C3EC80
:103090001FF0A6EC1DF00401480E826F92EC0AF0BE
:1030A00004017A0E826F92EC0AF004012C0E826FFA
:1030B00092EC0AF066C100F167C101F168C102F14A
:1030C00069C103F10101C3EC1FF0A6EC1DF004017E
:1030D000630E826F92EC0AF004012C0E826F92EC68
:1030E0000AF066C100F167C101F168C102F169C16E
:1030F00003F101010A0E046F000E056F000E066F4A
:10310000000E076F36EC1FF0000E046F120E056FF5
:10311000000E066F000E076F56EC1FF0C3EC1FF099
:103120002AC182F40401300E822792EC0AF02BC1EE
:1031300082F40401300E822792EC0AF02CC182F452
:103140000401300E822792EC0AF02DC182F40401B2
:10315000300E822792EC0AF02EC182F40401300E68
:10316000822792EC0AF02FC182F40401300E8227EC
:1031700092EC0AF030C182F40401300E822792EC06
:103180000AF004012E0E826F92EC0AF031C182F433
:103190000401300E822792EC0AF032C182F404015D
:1031A000300E822792EC0AF033C182F40401300E13
:1031B000822792EC0AF00401730E826F92EC0AF0FF
:1031C00004012C0E826F92EC0AF020EC20F059C121
:1031D00000F15AC101F189EC1AF00FB2F3EF18F0C7
:1031E0000FA025EF19F004012C0E826F92EC0AF06B
:1031F000200EF86EF76AF66A04010900F5CF82F432
:1032000092EC0AF00900F5CF82F492EC0AF0090082
:10321000F5CF82F492EC0AF00900F5CF82F492EC3B
:103220000AF00900F5CF82F492EC0AF00900F5CF1C
:1032300082F492EC0AF00900F5CF82F492EC0AF0E5
:103240000900F5CF82F492EC0AF09CEC0AF00F90A2
:103250005FEF19F00401630E826F92EC0AF0040133
:103260002C0E826F92EC0AF065EC19F004012C0E22
:10327000826F92EC0AF0D8EC19F004012C0E826FE8
:1032800092EC0AF054EC1AF004012C0E826F92ECCE
:103290000AF00101F80E006FCD0E016F660E026F8D
:1032A000030E036F7AEC19F004012C0E826F92EC7E
:1032B0000AF06AEC1AF09CEC0AF05FEF19F00301D7
:1032C000C26B079010926EEF1CF0D8900E0EA4EC1B
:1032D00007F0E8CF00F10F0EA4EC07F0E8CF01F102
:1032E000100EA4EC07F0E8CF02F1110EA4EC07F0E9
:1032F000E8CF03F10101000E046F000E056F010E0F
:10330000066F000E076F56EC1FF0C3EC1FF02AC1CA
:1033100082F40401300E822792EC0AF02BC182F471
:103320000401300E822792EC0AF02CC182F40401D1
:10333000300E822792EC0AF02DC182F40401300E87
:10334000822792EC0AF02EC182F40401300E82270B
:1033500092EC0AF02FC182F40401300E822792EC25
:103360000AF030C182F40401300E822792EC0AF098
:1033700031C182F40401300E822792EC0AF004017C
:103380002E0E826F92EC0AF032C182F40401300EEC
:10339000822792EC0AF033C182F40401300E8227B6
:1033A00092EC0AF004016D0E826F92EC0AF01200AA
:1033B000120EA4EC07F0E8CF00F1130EA4EC07F016
:1033C000E8CF01F1140EA4EC07F0E8CF02F1150EDE
:1033D000A4EC07F0E8CF03F101010A0E046F000E20
:1033E000056F000E066F000E076F36EC1FF0000E23
:1033F000046F120E056F000E066F000E076F56EC7D
:103400001FF0C3EC1FF02AC182F40401300E8227A2
:1034100092EC0AF02BC182F40401300E822792EC68
:103420000AF02CC182F40401300E822792EC0AF0DB
:103430002DC182F40401300E822792EC0AF02EC1D5
:1034400082F40401300E822792EC0AF02FC182F43C
:103450000401300E822792EC0AF030C182F404019C
:10346000300E822792EC0AF004012E0E826F92EC4D
:103470000AF031C182F40401300E822792EC0AF086
:1034800032C182F40401300E822792EC0AF033C17B
:1034900082F40401300E822792EC0AF00401730ECC
:1034A000826F92EC0AF012000A0EA4EC07F0E8CF4B
:1034B00000F10B0EA4EC07F0E8CF01F10C0EA4EC28
:1034C00007F0E8CF02F10D0EA4EC07F0E8CF03F10E
:1034D00089EF1AF0060EA4EC07F0E8CF00F1070E12
:1034E000A4EC07F0E8CF01F1080EA4EC07F0E8CF58
:1034F00002F1090EA4EC07F0E8CF03F189EF1AF00E
:10350000010120EC20F0078457C100F158C101F1FE
:1035100007940101E80E046F800E056F000E066F20
:10352000000E076F36EC1FF0000E046F040E056FDF
:10353000000E066F000E076F56EC1FF0880E046F2A
:10354000130E056F000E066F000E076F25EC1FF0BF
:103550000A0E046F000E056F000E066F000E076F57
:1035600056EC1FF0C3EC1FF001012967BDEF1AF004
:103570000401200E826FC0EF1AF004012D0E826F3D
:1035800092EC0AF030C182F40401300E822792ECF2
:103590000AF031C182F40401300E822792EC0AF065
:1035A00032C182F40401300E822792EC0AF0040149
:1035B0002E0E826F92EC0AF033C182F40401300EB9
:1035C000822792EC0AF00401430E826F92EC0AF01B
:1035D000120087C32AF188C32BF189C32CF18AC357
:1035E0002DF18BC32EF18CC32FF18DC330F18EC31F
:1035F00031F190C332F191C333F10101296B6EECCB
:1036000020F0E5EC1FF00101000E046F000E056FC5
:10361000010E066F000E076F36EC1FF00E0E0C6EDB
:1036200000C10BF08DEC07F00F0E0C6E01C10BF01A
:103630008DEC07F0100E0C6E02C10BF08DEC07F054
:10364000110E0C6E03C10BF08DEC07F004017A0E25
:10365000826F92EC0AF004012C0E826F92EC0AF059
:103660000401350E826F92EC0AF004012C0E826F79
:1036700092EC0AF065EC19F06DEF15F087C32AF1B2
:1036800088C32BF189C32CF18AC32DF18BC32EF192
:103690008CC32FF18DC330F18EC331F190C332F161
:1036A00091C333F10101296B6EEC20F0E5EC1FF0C2
:1036B000880E046F130E056F000E066F000E076F65
:1036C0002AEC1FF0000E046F040E056F000E066F4B
:1036D000000E076F36EC1FF00101E80E046F800E3C
:1036E000056F000E066F000E076F56EC1FF00A0EF6
:1036F0000C6E00C10BF08DEC07F00B0E0C6E01C1CF
:103700000BF08DEC07F00C0E0C6E02C10BF08DEC83
:1037100007F00D0E0C6E03C10BF08DEC07F00401E9
:103720007A0E826F92EC0AF004012C0E826F92ECFA
:103730000AF00401360E826F92EC0AF004012C0E9E
:10374000826F92EC0AF054EC1AF06DEF15F087C31B
:103750002AF188C32BF189C32CF18AC32DF18BC3C5
:103760002EF18CC32FF18DC330F18FC331F190C393
:1037700032F191C333F101016EEC20F0E5EC1FF062
:10378000000E046F120E056F000E066F000E076F1D
:1037900036EC1FF001010A0E046F000E056F000EDB
:1037A000066F000E076F56EC1FF0120E0C6E00C174
:1037B0000BF08DEC07F0130E0C6E01C10BF08DECCD
:1037C00007F0140E0C6E02C10BF08DEC07F0150E15
:1037D0000C6E03C10BF08DEC07F004017A0E826FC2
:1037E00092EC0AF004012C0E826F92EC0AF00401B4
:1037F000370E826F92EC0AF004012C0E826F92EC6D
:103800000AF0D8EC19F06DEF15F087C32AF188C3E0
:103810002BF189C32CF18AC32DF18BC32EF18CC3FC
:103820002FF18DC330F18EC331F190C332F191C3CA
:1038300033F10101296B6EEC20F0E5EC1FF0880EEE
:10384000046F130E056F000E066F000E076F2AEC53
:103850001FF0000E046F040E056F000E066F000EC1
:10386000076F36EC1FF00101E80E046F800E056F44
:10387000000E066F000E076F56EC1FF0060E0C6E62
:1038800000C10BF08DEC07F0070E0C6E01C10BF0C0
:103890008DEC07F0080E0C6E02C10BF08DEC07F0FA
:1038A000090E0C6E03C10BF08DEC07F004017A0ECB
:1038B000826F92EC0AF004012C0E826F92EC0AF0F7
:1038C0000401380E826F92EC0AF004012C0E826F14
:1038D00092EC0AF06AEC1AF06DEF15F081A82CEF6B
:1038E0001DF007A8E5EF1CF00101800E006F1A0E15
:1038F000016F060E026F000E036F4BC104F14CC145
:1039000005F14DC106F14EC107F125EC1FF003BFD3
:103910002CEF1DF0A0EC1DF04BC100F14CC101F1EA
:103920004DC102F14EC103F1078232EC1EF018C105
:1039300004F119C105F11AC106F11BC107F1F80E16
:10394000006FCD0E016F660E026F030E036F25EC44
:103950001FF00E0E0C6E00C10BF08DEC07F00F0E79
:103960000C6E01C10BF08DEC07F0100E0C6E02C155
:103970000BF08DEC07F0110E0C6E03C10BF08DEC0B
:1039800007F00784010120EC20F057C100F158C175
:1039900001F107940A0E0C6E00C10BF08DEC07F0DC
:1039A0000B0E0C6E01C10BF08DEC07F00C0E0C6EC3
:1039B00002C10BF08DEC07F00D0E0C6E03C10BF085
:1039C0008DEC07F007982CEF1DF007AA2CEF1DF0E7
:1039D0000784010120EC20F057C100F158C101F12A
:1039E0000794060E0C6E00C10BF08DEC07F0070E6D
:1039F0000C6E01C10BF08DEC07F0080E0C6E02C1CD
:103A00000BF08DEC07F0090E0C6E03C10BF08DEC82
:103A100007F0078462C100F163C101F164C102F1E2
:103A200065C103F10794120E0C6E00C10BF08DEC12
:103A300007F0130E0C6E01C10BF08DEC07F0140EA5
:103A40000C6E02C10BF08DEC07F0150E0C6E03C16D
:103A50000BF08DEC07F0079A0401805181197F0B60
:103A60000BE09EA809D014EE00F081517F0BE126F7
:103A7000E750812B0F01AD6E05012F51010A13E0B4
:103A800081AA53EF1DF005012F51000A0AE00FB87B
:103A900053EF1DF00501306753EF1DF00FB853EFE2
:103AA0001DF0FFEF26F081B868EF1DF03EEC21F02D
:103AB00005012F51020A02E068EF1DF05C2F68EF4C
:103AC0001DF05BC55CF50501010E306F3C0E316FDA
:103AD00000EF0AF018C100F119C101F11AC102F199
:103AE0001BC103F1000E046F000E056F010E066F7F
:103AF000000E076F56EC1FF029A195EF1DF0205125
:103B0000D8B495EF1DF018C100F119C101F11AC127
:103B100002F11BC103F1000E046F000E056F0A0EC7
:103B2000066F000E076F56EC1FF0120001010451E2
:103B3000001305510113065102130751031312001C
:103B40000101186B196B1A6B1B6B12002AC182F4EE
:103B50000401300E822792EC0AF02BC182F404019A
:103B6000300E822792EC0AF02CC182F40401300E50
:103B7000822792EC0AF02DC182F40401300E8227D4
:103B800092EC0AF02EC182F40401300E822792ECEE
:103B90000AF02FC182F40401300E822792EC0AF061
:103BA00030C182F40401300E822792EC0AF031C158
:103BB00082F40401300E822792EC0AF032C182F4C2
:103BC0000401300E822792EC0AF033C182F4040122
:103BD000300E822792EC0AF012002FC182F4040109
:103BE000300E822792EC0AF030C182F40401300ECC
:103BF000822792EC0AF031C182F40401300E822750
:103C000092EC0AF032C182F40401300E822792EC69
:103C10000AF033C182F40401300E822792EC0AF0DC
:103C20001200060E116E060E126E060E136E112E87
:103C300017EF1EF0122E17EF1EF0132E17EF1EF0C7
:103C40008B84020E116E020E126E020E136E112E76
:103C500027EF1EF0122E27EF1EF0132E27EF1EF077
:103C60008B9412000101005305E1015303E102535B
:103C700001E1002BF5EC1EF020EC20F03951006F33
:103C80003A51016F420E046F4B0E056F000E066F26
:103C9000000E076F36EC1FF000C104F101C105F101
:103CA00002C106F103C107F118C100F119C101F108
:103CB0001AC102F11BC103F107B263EF1EF02AEC37
:103CC0001FF065EF1EF025EC1FF000C118F101C1D7
:103CD00019F102C11AF103C11BF1120020EC20F00E
:103CE00059C100F15AC101F1060EA4EC07F0E8CF6A
:103CF00004F1070EA4EC07F0E8CF05F1080EA4ECE0
:103D000007F0E8CF06F1090EA4EC07F0E8CF07F1C1
:103D100025EC1FF000C124F101C125F102C126F1FB
:103D200003C127F1290E046F000E056F000E066F08
:103D3000000E076F36EC1FF0EE0E046F430E056F9A
:103D4000000E066F000E076F2AEC1FF024C104F16D
:103D500025C105F126C106F127C107F136EC1FF098
:103D600000C11CF101C11DF102C11EF103C11FF10F
:103D7000120EA4EC07F0E8CF04F1130EA4EC07F048
:103D8000E8CF05F1140EA4EC07F0E8CF06F1150E0C
:103D9000A4EC07F0E8CF07F10D0E006F000E016FE5
:103DA000000E026F000E036F36EC1FF0180E046F4A
:103DB000000E056F000E066F000E076F56EC1FF029
:103DC0001CC104F11DC105F11EC106F11FC107F19F
:103DD0002AEC1FF06A0E046F2A0E056F000E066FA4
:103DE000000E076F25EC1FF01200BF0EFA6E200EBA
:103DF0003A6F396BD8900037013702370337D8B0A4
:103E000006EF1FF03A2FFBEF1EF039073A07035376
:103E1000D8B412000331070B80093F6F03390F0B31
:103E2000010F396F80EC5FF0406F390580EC5FF077
:103E3000405D405F396B3F33D8B0392739333FA9F4
:103E40001BEF1FF0405139271200010145EC20F013
:103E5000D8B01200010103510719346F08EC20F0AB
:103E6000D8900751031934AF800F12000101346B51
:103E70002CEC20F0D8A042EC20F0D8B0120017ECC7
:103E800020F020EC20F01F0E366F58EC20F00B35A0
:103E9000D8B008EC20F0D8A00335D8B01200362FE7
:103EA00045EF1FF034B12FEC20F012000101346B0C
:103EB00004510511061107110008D8A02CEC20F0C0
:103EC000D8A042EC20F0D8B01200086B096B0A6B46
:103ED0000B6B58EC20F01F0E366F58EC20F007519A
:103EE0000B5DD8A480EF1FF006510A5DD8A480EFC7
:103EF0001FF00551095DD8A480EF1FF00451085D43
:103F0000D8A093EF1FF00451085F0551D8A0053DDC
:103F1000095F0651D8A0063D0A5F0751D8A0073DAA
:103F20000B5FD8900081362F6DEF1FF034B12FEC6E
:103F300020F0346B2CEC20F0D8905CEC20F0075192
:103F40000B5DD8A4B0EF1FF006510A5DD8A4B0EF06
:103F50001FF00551095DD8A4B0EF1FF00451085DB2
:103F6000D8A0BFEF1FF0003FBFEF1FF0013FBFEF32
:103F70001FF0023FBFEF1FF0032BD8B4120034B183
:103F80002FEC20F012000101346B2CEC20F0D8B0A3
:103F9000120061EC20F0200E366F00370137023737
:103FA000033711EE33F00A0E376FE7360A0EE75C7F
:103FB000D8B0E76EE552372FD5EF1FF0362FCDEF93
:103FC0001FF034B12981D890120001010A0E346F1C
:103FD000200E366F11EE29F03451376F0A0ED8904B
:103FE000E652D8B0E726E732372FF0EF1FF0033361
:103FF000023301330033362FEAEF1FF0E750FF0F93
:10400000D8A00335D8B0120029B12FEC20F012004F
:10401000045100270551D8B0053D01270651D8B0FD
:10402000063D02270751D8B0073D03271200005173
:10403000086F0151096F02510A6F03510B6F120093
:104040000101006B016B026B036B12000101046B39
:10405000056B066B076B12000335D8A012000351E5
:10406000800B001F011F021F031F003F3FEF20F0C6
:10407000013F3FEF20F0023F3FEF20F0032B342BB6
:10408000032512000735D8A012000751800B041F2A
:10409000051F061F071F043F55EF20F0053F55EF92
:1040A00020F0063F55EF20F0072B342B0725120098
:1040B0000037013702370337083709370A370B371C
:1040C00012000101296B2A6B2B6B2C6B2D6B2E6B55
:1040D0002F6B306B316B326B336B120001012A5145
:1040E0000F0B2A6F2B510F0B2B6F2C510F0B2C6FBB
:1040F0002D510F0B2D6F2E510F0B2E6F2F510F0BBC
:104100002F6F30510F0B306F31510F0B316F325118
:104110000F0B326F33510F0B336F12008984000E77
:10412000C76E220EC66E9E96C69E000EC96EFF0E0C
:104130009EB602D0E82EFCD79E96C69E000EC96E93
:10414000FF0E9EB602D0E82EFCD7C9CFABF59E96E7
:10415000C69E000EC96EFF0E9EB602D0E82EFCD79A
:10416000C9CFACF59E96C69E000EC96EFF0E9EB6D8
:1041700002D0E82EFCD7C9CFADF59E96C69E000EA4
:10418000C96EFF0E9EB602D0E82EFCD7C9CFAEF5A1
:104190009E96C69E000EC96EFF0E9EB602D0E82EF9
:1041A000FCD7C9CFAFF59E96C69E000EC96EFF0E16
:1041B0009EB602D0E82EFCD7C9CFB0F59E96C69E1B
:1041C000000EC96EFF0E9EB602D0E82EFCD7C9CFF6
:1041D000B1F5899441EC23F012008984000EC76E7A
:1041E000220EC66E9E96C69E800EC96EFF0E9EB6AD
:1041F00002D0E82EFCD79E96C69EABC5C9FFFF0E27
:104200009EB602D0E82EFCD79E96C69EACC5C9FFCE
:10421000FF0E9EB602D0E82EFCD79E96C69EADC578
:10422000C9FFFF0E9EB602D0E82EFCD79E96C69E12
:10423000AEC5C9FFFF0E9EB602D0E82EFCD79E96F3
:10424000C69EAFC5C9FFFF0E9EB602D0E82EFCD7B2
:104250009E96C69EB0C5C9FFFF0E9EB602D0E82E40
:10426000FCD79E96C69EB1C5C9FFFF0E9EB602D072
:10427000E82EFCD7899441EC23F012008984000ECB
:10428000C76E220EC66E9E96C69E070EC96EFF0EA4
:104290009EB602D0E82EFCD79E96C69E000EC96E32
:1042A000FF0E9EB602D0E82EFCD7C9CFABF59E9686
:1042B000C69E000EC96EFF0E9EB602D0E82EFCD739
:1042C000C9CFACF59E96C69E000EC96EFF0E9EB677
:1042D00002D0E82EFCD7C9CFADF59E96C69E000E43
:1042E000C96EFF0E9EB602D0E82EFCD7C9CFAEF540
:1042F000899441EC23F08984000EC76E220EC66EAD
:104300009E96C69E0F0EC96EFF0E9EB602D0E82E78
:10431000FCD79E96C69E000EC96EFF0E9EB602D0BA
:10432000E82EFCD7C9CFB3F5899441EC23F01200F5
:104330008984000EC76E220EC66E9E96C69E870E9C
:10434000C96EFF0E9EB602D0E82EFCD79E96C69E82
:10435000ABC5C9FFFF0E9EB602D0E82EFCD79E96D5
:10436000C69EACC5C9FFFF0E9EB602D0E82EFCD794
:104370009E96C69EADC5C9FFFF0E9EB602D0E82E22
:10438000FCD79E96C69EAEC5C9FFFF0E9EB602D054
:10439000E82EFCD7899441EC23F089849E96C69E32
:1043A0008F0EC96EFF0E9EB602D0E82EFCD79E96E9
:1043B000C69EB3C5C9FFFF0E9EB602D0E82EFCD73D
:1043C000899441EC23F012008984000EC76E220EFE
:1043D000C66E9E96C69E870EC96EFF0E9EB602D012
:1043E000E82EFCD79E96C69E000EC96EFF0E9EB6A6
:1043F00002D0E82EFCD79E96C69E800EC96EFF0E98
:104400009EB602D0E82EFCD79E96C69E800EC96E40
:10441000FF0E9EB602D0E82EFCD79E96C69E800E5A
:10442000C96EFF0E9EB602D0E82EFCD7899441ECEF
:1044300023F089849E96C69E8F0EC96EFF0E9EB68F
:1044400002D0E82EFCD79E96C69E010EC96EFF0EC6
:104450009EB602D0E82EFCD7899441EC23F01200DE
:104460008984000EC76E220EC66E9E96C69E870E6B
:10447000C96EFF0E9EB602D0E82EFCD79E96C69E51
:10448000000EC96EFF0E9EB602D0E82EFCD79E9697
:10449000C69E000EC96EFF0E9EB602D0E82EFCD757
:1044A0009E96C69E800EC96EFF0E9EB602D0E82E66
:1044B000FCD79E96C69E800EC96EFF0E9EB602D099
:1044C000E82EFCD7899441EC23F089849E96C69E01
:1044D0008F0EC96EFF0E9EB602D0E82EFCD79E96B8
:1044E000C69E010EC96EFF0E9EB602D0E82EFCD706
:1044F000899441EC23F012008984000EC76E220ECD
:10450000C66E9E96C69E8F0EC96EFF0E9EB602D0D8
:10451000E82EFCD741EC23F09E96C69E810EC96E14
:10452000FF0E9EB602D0E82EFCD7899441EC23F012
:104530008984000EC76E220EC66E9E96C69E8F0E92
:10454000C96EFF0E9EB602D0E82EFCD741EC23F0D8
:104550009E96C69E010EC96EFF0E9EB602D0E82E34
:10456000FCD7899441EC23F089849E96C69E910ED7
:10457000C96EFF0E9EB602D0E82EFCD741EC23F0A8
:104580009E96C69EA50EC96EFF0E9EB602D0E82E60
:10459000FCD7899441EC23F012008984000EC76E89
:1045A000220EC66E9E96C69E8F0EC96EFF0E9EB6DA
:1045B00002D0E82EFCD741EC23F09E96C69E810ED9
:1045C000C96EFF0E9EB602D0E82EFCD7899441EC4E
:1045D00023F012008984000EC76E220EC66E9E96CE
:1045E000C69E8F0EC96EFF0E9EB602D0E82EFCD777
:1045F00041EC23F09E96C69E010EC96EFF0E9EB63C
:1046000002D0E82EFCD7899441EC23F01200898473
:10461000000EC76E220EC66E9E96C69E910EC96E85
:10462000FF0E9EB602D0E82EFCD741EC23F09E96FA
:10463000C69EA50EC96EFF0E9EB602D0E82EFCD710
:10464000899441EC23F012008984000EC76E220E7B
:10465000C66E9E96C69E910EC96EFF0E9EB602D085
:10466000E82EFCD741EC23F09E96C69E000EC96E44
:10467000FF0E9EB602D0E82EFCD7899441EC23F0C1
:104680001200050EE82EFED712000501256B266BE1
:10469000276B286B899A400EC76E200EC66E9E96B9
:1046A000C69E030EC96EFF0E9EB602D0E82EFCD742
:1046B0009E96C69E27C5C9FFFF0E9EB602D0E82E65
:1046C000FCD79E96C69E26C5C9FFFF0E9EB602D099
:1046D000E82EFCD79E96C69E25C5C9FFFF0E9EB646
:1046E00002D0E82EFCD79E96C69EC952FF0E9EB6FB
:1046F00002D0E82EFCD7898A0F01C950FF0A01E1D8
:10470000120005012E51130A05E005012E51170A6A
:104710000CE012000501F00E256FFF0E266F0F0E44
:10472000276F000E286F9EEF23F00501F00E256F16
:10473000FF0E266FFF0E276F000E286F899A400E1E
:10474000C76E200EC66E9E96C69E030EC96EFF0EE5
:104750009EB602D0E82EFCD79E96C69E27C5C9FFFE
:10476000FF0E9EB602D0E82EFCD79E96C69E26C5AA
:10477000C9FFFF0E9EB602D0E82EFCD79E96C69EBD
:1047800025C5C9FFFF0E9EB602D0E82EFCD79E9627
:10479000C69EC952FF0E9EB602D0E82EFCD7898A6B
:1047A0000F01C950FF0A1DE005012E51130A05E053
:1047B00005012E51170A0BE012000501000E256FAE
:1047C000000E266F100E276F000E286F12000501D5
:1047D000000E256F000E266F000E276F010E286F4A
:1047E00012000501256B266B276B286B05012E51E6
:1047F000130A05E005012E51170A0CE0120005010D
:10480000000E216F000E226F080E236F000E246F22
:1048100013EF24F00501000E216F000E226F800EB1
:10482000236F000E246F21C500F122C501F123C5BD
:1048300002F124C503F125C504F126C505F127C5FC
:1048400006F128C507F196EC1DF000C125F501C160
:1048500026F502C127F503C128F5899A400EC76ED7
:10486000200EC66E9E96C69E030EC96EFF0E9EB6A5
:1048700002D0E82EFCD79E96C69E27C5C9FFFF0E24
:104880009EB602D0E82EFCD79E96C69E26C5C9FFCE
:10489000FF0E9EB602D0E82EFCD79E96C69E25C57A
:1048A000C9FFFF0E9EB602D0E82EFCD79E96C69E8C
:1048B000C952FF0E9EB602D0E82EFCD7898AC95095
:1048C000FF0A08E104C125F505C126F506C127F553
:1048D00007C128F5D890050124332333223321332F
:1048E0002151F00B216F21677DEF24F022677DEFCE
:1048F00024F023677DEF24F0246713EF24F00501F3
:10490000100E2527E86A2623E86A2723E86A282369
:104910001200E86A05012E51130A06E005012E5126
:10492000170A0BE0020E120005012851000A03E1EC
:104930002751F00B07E0010E120005012851000A73
:1049400001E0010E120029C500F12AC501F12BC5B5
:1049500002F12CC503F125C504F126C505F127C5D3
:1049600006F128C507F125EC1FF003BF120089EC02
:1049700024F05FE1899A400EC76E200EC66E9E96A7
:10498000C69E060EC96EFF0E9EB602D0E82EFCD75C
:10499000898A899A9E96C69E020EC96EFF0E9EB6A1
:1049A00002D0E82EFCD79E96C69E27C5C9FFFF0EF3
:1049B0009EB602D0E82EFCD79E96C69E26C5C9FF9D
:1049C000FF0E9EB602D0E82EFCD79E96C69E25C549
:1049D000C9FFFF0E9EB602D0E82EFCD79E96C69E5B
:1049E000000EC96EFF0E9EB602D0E82EFCD7898A53
:1049F000899A9E96C69E050EC96EFF0E9EB602D07F
:104A0000E82EFCD79E96C69EC952FF0E9EB602D0D7
:104A1000E82EFCD7C9B002EF25F0898A0501100EF7
:104A20002527E86A2623E86A2723E86A2823A3EFD4
:104A300024F01200899A400EC76E200EC66E9E9614
:104A4000C69E060EC96EFF0E9EB602D0E82EFCD79B
:104A5000898A899A9E96C69EC70EC96EFF0E9EB61B
:104A600002D0E82EFCD7898A0501256B266B276BBF
:104A7000286B1200899A400EC76E200EC66E9E9655
:104A8000C69E050EC96EFF0E9EB602D0E82EFCD75C
:104A90009E96C69EC952FF0E9EB602D0E82EFCD747
:104AA000C9CF33F5898A1200899A400EC76E200E4D
:104AB000C66E9E96C69EB90EC96EFF0E9EB602D0F9
:104AC000E82EFCD7898A1200899A400EC76E200E04
:104AD000C66E9E96C69EAB0EC96EFF0E9EB602D0E7
:104AE000E82EFCD7898AFF0EE82EFED7120089EC4B
:104AF00024F0D8A41200899A400EC76E200EC66E0C
:104B00009E96C69E030EC96EFF0E9EB602D0E82E7C
:104B1000FCD79E96C69E27C5C9FFFF0E9EB602D043
:104B2000E82EFCD79E96C69E26C5C9FFFF0E9EB6F0
:104B300002D0E82EFCD79E96C69E25C5C9FFFF0E63
:104B40009EB602D0E82EFCD79E96C69EC952FF0E96
:104B50009EB602D0E82EFCD7898A0F01C950FF0A01
:104B6000D8A472EF26F00501FE0E336F8EEC20F014
:104B7000ABC534F5ACC535F5ADC536F5AEC537F5C5
:104B8000AFC538F5B0C539F5B1C53AF50784B6C13A
:104B900066F1B7C167F1B8C168F1B9C169F14BC13C
:104BA0004FF14CC150F14DC151F14EC152F157C1BD
:104BB00059F158C15AF197EC15F000C13BF501C10C
:104BC0003CF502C13DF503C13EF505015D67F0EF1F
:104BD00025F05E67F0EF25F05F67F0EF25F0606786
:104BE000F4EF25F001EF26F05DC504F15EC505F197
:104BF0005FC506F160C507F125EC1FF003BF72EF3A
:104C000026F059C13FF55AC140F5B5C541F5B6C5C5
:104C100042F507940501110E326F899A400EC76E56
:104C2000200EC66E9E96C69E060EC96EFF0E9EB6DE
:104C300002D0E82EFCD7898A899A9E96C69E020EDB
:104C4000C96EFF0E9EB602D0E82EFCD79E96C69E79
:104C500027C5C9FFFF0E9EB602D0E82EFCD79E9650
:104C6000C69E26C5C9FFFF0E9EB602D0E82EFCD711
:104C70009E96C69E25C5C9FFFF0E9EB602D0E82EA1
:104C8000FCD725EE33F0322F02D052EF26F09E965D
:104C9000C69EDECFC9FFFF0E9EB602D0E82EFCD71F
:104CA00043EF26F0898A899A9E96C69E050EC96EA4
:104CB000FF0E9EB602D0E82EFCD79E96C69EC95225
:104CC000FF0E9EB602D0E82EFCD7C9B05DEF26F0ED
:104CD000898A0501100E2527E86A2623E86A27231A
:104CE000E86A2823120021C500F122C501F123C57D
:104CF00002F124C503F1899A400EC76E200EC66EDC
:104D00009E96C69E0B0EC96EFF0E9EB602D0E82E72
:104D1000FCD79E96C69E02C1C9FFFF0E9EB602D06A
:104D2000E82EFCD79E96C69E01C1C9FFFF0E9EB617
:104D300002D0E82EFCD79E96C69E00C1C9FFFF0E8A
:104D40009EB602D0E82EFCD79E96C69EC952FF0E94
:104D50009EB602D0E82EFCD725EE33F00501100EEA
:104D6000326F9E96C69EC952FF0E9EB602D0E82EA6
:104D7000FCD7C9CFDEFF322FB1EF26F0898A1200AF
:104D8000899A400EC76E200EC66E9E96C69E900EE5
:104D9000C96EFF0E9EB602D0E82EFCD79E96C69E28
:104DA000000EC96EFF0E9EB602D0E82EFCD79E966E
:104DB000C69E000EC96EFF0E9EB602D0E82EFCD72E
:104DC0009E96C69E000EC96EFF0E9EB602D0E82EBD
:104DD000FCD79E96C69EC952FF0E9EB602D0E82E04
:104DE000FCD7C9CF2DF59E96C69EC952FF0E9EB622
:104DF00002D0E82EFCD7C9CF2EF5898A120011EC1B
:104E00001EF0B5C5E8FFD70802E311EC1EF0B5C5EA
:104E1000E8FFC80802E311EC1EF0B5C5E8FFB908C9
:104E200002E311EC1EF0B5C5E8FFAA0802E311EC9D
:104E30001EF0B5C5E8FF9B0802E311EC1EF03EEC46
:104E400021F054EC25F0F29CF29E8B94C69AC2900D
:104E50009482948C720ED36ED3A4FED789968A90D6
:104E60009390FF0EE8CF00F0E82EFED7002EFCD77F
:104E70008150F294F29A9E909D909E929D92F2980B
:0C4E8000F292F290F286F28E0300FF0026
:10BF0000E844F926000C160C2B0C3F0C520C640C68
:10BF1000760C860C960CA50CB30CC10CCF0CDC0C6B
:06BF2000E80CF40C000C1B
:00000001FF
